:020000040000FA
:0400000080311D2806
:08000800200020002008A400E4
:100010002108A5002208A6002308A7009331322B4F
:100020000830AA000310A20D0310A00D031C1A280B
:100030002108A207AA0B12280800DA286D08200060
:10004000BD0021006E082000BE0008000310200043
:100050003E0C2200A10020003D0C2200A000031055
:10006000A10CA00C200820003D062200A2002108BF
:1000700020003E062200A300031020003E0C2200B8
:10008000A50020003D0C2200A4000310A50CA40C28
:100090000310A50CA40C24082206A600250823069C
:1000A000A700031020003E0C2200A90020003D0CF8
:1000B0002200A80004302000A00003102200A90C98
:1000C000A80C2000A00B5D28220028082606AA0004
:1000D00029082706AB0001302A052100EB00EC01BE
:1000E000031020003E0C2200A10020003D0C220045
:1000F000A000003021006B1880302200A201A30074
:10010000220820042000BD00220023082104200032
:10011000BE000800262020003D08A0003E08A100E7
:1001200008002620E13020003D02A000AC303E0255
:1001300020048031031D9E28003008003E0808007E
:100140002100241091131110013020009800990112
:100150008B170B1708002100241CB328FF30200048
:10016000A000A100080020001608A0001708A100A8
:1001700008003B0896003C0897002100241020004E
:10018000111021001114080021002410200011106A
:100190002100111008002000111CD128C4202000CB
:1001A00011152408A0002508A1002608A200270890
:1001B000A300090021008E1683314E2B2000C501BB
:1001C00021002411A411C420F030250013050438A7
:1001D00093002100A4132000111121001115080023
:1001E000DE2021002412A4120B178B170800813186
:1001F0002100241E06292510A418251420004708D4
:10020000C800210024122000201408002000201023
:100210000800A41E16292510A4182514200047083C
:10022000C8002100A4122000201408002000201083
:10023000080080312000111DCB28111181312100CF
:10024000A41F2429A4132529A417A41F2D29F030A5
:1002500025001305053893003229F03025001305D9
:10026000043893008031AB2020002008C30021080F
:10027000C400BB01BC018031B92020004508813198
:10028000031D46290130C5008031CB284503031DDD
:10029000902914304402031D4F29D0304302B51178
:1002A000031D0318B51522304402031D5929B0302F
:1002B00043023512031D031C3516B516B519351E3C
:1002C000B512B51E6F29210024172000BF01C001FF
:1002D000C101C201C6010230C50083312D2B3A3065
:1002E0004402031D7529403043023513031D0318D2
:1002F00035176C304402031D7F2938304302B51393
:10030000031D031CB5173614351BB51F3610361CDC
:100310008C290330C5008E298031DE208031CB2826
:10032000023045028231031D272A143044028131F4
:10033000031D9C29D03043023611031D03183615C6
:1003400022304402031DA629B0304302B611031D1A
:10035000031CB61536163619B61D3612361EC429BC
:100360002100241FC2292000C60A0310BF0DC00DA2
:10037000C10DC20D2100A41FBF2920003F14210080
:100380002413EC292417EC2929304402031DCA291F
:10039000B0304302B612031D0318B61645304402AE
:1003A000031DD429603043023613031D031C361786
:1003B000B617B61A361FB613B61FEA29C60A0310B7
:1003C000BF0DC00DC10DC20D2100A41FEC292000DE
:1003D0003F14EC298031DE200D30200046028031B0
:1003E000031DCB28AD0110304005AE00AF01B001B8
:1003F0002D082E042F04300482310319232AB10161
:1004000008304005B200B301B401310832043304AE
:1004100034042100A4140319A41007302000C005DF
:10042000C101C2013F303F05C700210024159F30A4
:100430002000BB00BA30BC008031B920053020005C
:10044000C5008031CB288031DE208031CB280330BD
:100450004502031D552A13304402031D312A68301A
:1004600043023712031D0318371624304402031DBC
:100470003B2A10304302B712031D031CB71637176F
:10048000371AB71E3713371F512A210024172000AF
:10049000BF01C001C101C201C6010430C5008031E5
:1004A000CB288031DE208031CB28043045028331D7
:1004B000031D202B093044028231031D612AB03014
:1004C00043023810031D0318381412304402031D70
:1004D0006B2A08304302B810031D031CB8143815EA
:1004E0003818B81C3811381D892A2100241F872A82
:1004F0002000C60A0310BF0DC00DC10DC20D2100A2
:10050000A41B842A20003F1421002413DD2A241771
:10051000DD2A13304402031D8F2A6830430238124B
:10052000031D0318381624304402031D992A103085
:100530004302B812031D031CB8163817381AB81E28
:100540003813381FB32A053046020319DD2AC60ABC
:100550000310BF0DC00DC10DC20D2100A41BDD2A6B
:1005600020003F14DD2A1D304402031DB92A20302B
:100570004302B910031D0318B91436304402031D99
:10058000C32A183043023911031D031C3915B9154C
:10059000B918391DB911B91DDB2AC60A0310BF0DE0
:1005A000C00DC10DC20D2100A41BD82A20003F148C
:1005B00021002413DD2A8031DE2015302000460280
:1005C0008031031DCB28AD01AE0110304105AF00D5
:1005D000B0012D082E042F043004833103191C2B85
:1005E0004108A0004208A100A201A3010310A10C30
:1005F000A00C2008B100AD01AE0101304105AF00F3
:10060000B0012D082E042F0430042100A414031976
:10061000A4102000C101C2013F08C7002100A41599
:10062000EF302000BB00DB30BC008031B92005304A
:100630002000C5008031CB288031DE208031CB28DE
:10064000053045028031031DCB28210024122419D6
:100650002416A412A419A416DE208031CB28210070
:10066000EA002300910095131513151413080800D0
:10067000E8002300910021006908230093009513EE
:10068000151315158B1355309600AA309600951446
:100690008B171511951C4D2B4A2B08000C108C1034
:1006A0000C110E108E100E118E110E128C12933131
:1006B000062B20001C1187309C05FC301C050138DE
:1006C0009C006F309B0091102100911420001C159C
:1006D0000B178B17080028001711873017053038C3
:1006E0009700FC30170503389700FF309600200074
:1006F000931021009314280017150B178B1708006F
:1007000081312000911C192991104A088331031965
:100710008B2BCA038D2B22000C1420004F080319C9
:10072000932BCF03952B22008C142000540803191F
:100730009B2BD4039D2B22000C1520005908031974
:10074000A32BD903A52B22000E1420005E08031949
:10075000AB2BDE03AD2B22008E142000630803199F
:10076000B32BE303B52B22000E15200068080319F4
:10077000BB2BE803BD2B22008E1520006D0803194A
:10078000C32BED03C52B22000E162000720803199F
:10079000CC2BF2038131192922008C1681311929C1
:1007A0002000931C802B93104908CA004A080319A3
:1007B000DB2B22000C1020004E08CF004F0803193D
:1007C000E32B22008C1020005308D4005408031996
:1007D000EB2B22000C1120005808D90059080319EE
:1007E000F32B22000E1020005D08DE005E0883312E
:1007F0000319FC2B22008E1020006208E30063081E
:1008000084310319052C22000E1120006708E8002E
:10081000680803190D2C22008E1120006C08ED00D1
:100820006D080319152C22000E1220007108F20029
:10083000720883310319802B22008C12802B210037
:10084000E50165082000A0000F30A10080311020D4
:10085000200022082100E600493084008501660856
:1008600084078001200022082100E600660AE700D4
:100870004930840085016708840780012000220830
:100880002100E60002306607E70049308400850158
:10089000670884078001200022082100E600033059
:1008A0006607E700493084008501670884078001F6
:1008B000200022082100E60004306607E7004930E6
:1008C0008400850167088407800120002208210038
:1008D000E60005306607E7004930840085016708B7
:1008E00084078001200022082100E6000630660708
:1008F000E7004930840085016708840780012000F3
:1009000022082100E60007306607E700493084002E
:100910008501670884078001200022082100E60085
:1009200008306607E70049308400850167088407BE
:100930008001200022082100E60009306607E70058
:10094000493084008501670884078001200022085F
:100950002100E6000A306607E7004930840085017F
:10096000670884078001200022082100E6000B3080
:100970006607E70049308400850167088407800125
:10098000200022082100E6000C306607E70049300D
:100990008400850167088407800120002208210067
:1009A000E6000D306607E7004930840085016708DE
:1009B00084078001200022082100E6000E3066072F
:1009C000E700493084008501670884078001E50A53
:1009D000033065028431031D212C080020004B08E0
:1009E00021006214031D6210200050082100E2144F
:1009F000031DE21062156218E21C62112000550806
:100A00002100E215031DE21162166219E21D621255
:100A100020005A082100E216031DE2126217621A32
:100A2000E21E621320005F082100E217031DE2139B
:100A30006314621BE21F6310200064082100E314AA
:100A4000031DE31063156318E31C6311200069089C
:100A50002100E315031DE31163166319E31D6312FF
:100A600020006E082100E316031DE3126317631ACA
:100A7000E31E6313200073082100E317031DE31333
:100A80006414631BE31F6410853164184A2D200031
:100A900020100800200020140800D9002000C90000
:100AA00021005A082000CE0021005B082000D3005E
:100AB00021005C082000D80021005D082000DD0036
:100AC00021005E082000E20021005F082000E7000E
:100AD000210060082000EC00210061082000F100E6
:100AE0000800D00150082000A0000F30A100803184
:100AF0001020200022082100D10002305107D2002E
:100B000049308400850152088407000887310319A1
:100B10000B2F4930840085015208840703300002FE
:100B2000853103199C2D49308400850152088407C2
:100B300004300002031D9E2D87310B2F49308400A5
:100B400085015208840700038631031D552E500885
:100B50002000A0000F30A1008031102020002208CA
:100B60002100D10004305107D200493084008501B2
:100B700052088407000885310319E62D500820002B
:100B8000A0000F30A1008031102020002208210099
:100B9000D30004305307D400200022082100D500E0
:100BA00004305507D6004930840085015608840773
:100BB00000082000A000493084008501210054086D
:100BC000840720002003800087310B2F500820006D
:100BD000A0000F30A1008031102020002208210049
:100BE000D10004305107D2004930840085015208F9
:100BF000840777088000200022082100D10020000F
:100C000022082100D20003305207D300493084006B
:100C100085015108840700082000A00049308400A5
:100C20008501210053088407200020080002863136
:100C300003193D2E210050082000A0000F30A10014
:100C400080311020200022082100D400200022083A
:100C50002100D5004930840085015508840700082B
:100C60002000A00049308400850121005408840739
:100C70002000200A80008631532E210050082000D9
:100C8000A0000F30A1008031102020002208210098
:100C9000D10002305107D20049308400850152084A
:100CA00084070330800087310B2F49308400850191
:100CB00052088407023000028731031D0B2F5008B1
:100CC0002000A0000F30A100803110202000220859
:100CD0002100D10004305107D20049308400850141
:100CE000520884070008863103199E2E5008200000
:100CF000A0000F30A1008031102020002208210028
:100D0000D30004305307D400200022082100D5006E
:100D100004305507D6004930840085015608840701
:100D200000082000A00049308400850121005408FB
:100D3000840720002003800087310B2F50082000FB
:100D4000A0000F30A10080311020200022082100D7
:100D5000D10004305107D200493084008501520887
:100D6000840777088000200022082100D10020009D
:100D700022082100D20003305207D30049308400FA
:100D800085015108840700082000A0004930840034
:100D900085012100530884072000200800028631C5
:100DA0000319F52E210050082000A0000F30A100EB
:100DB00080311020200022082100D40020002208C9
:100DC0002100D500493084008501550884070008BA
:100DD0002000A000493084008501210054088407C8
:100DE00020002003800087310B2F210050082000B5
:100DF000A0000F30A1008031102020002208210027
:100E0000D10002305107D2004930840085015208D8
:100E1000840704308000200022082100D100073020
:100E20005107D20049308400850152088407000828
:100E300088310319AE28493084008501520884079F
:100E400003300002873103192E2F493084008501B9
:100E50005208840704300002031D302F8831AE2869
:100E6000493084008501520884070003031DEF2FD9
:100E700050082000A0000F30A10080311020200079
:100E800022082100D10009305107D20049308400E6
:100E9000850152088407000887310319772F50080D
:100EA0002000A0000F30A100803110202000220877
:100EB0002100D30009305307D4002000220821006C
:100EC000D50009305507D600493084008501560801
:100ED000840700082000A00049308400850121001B
:100EE000540884072000200380008831AE28500871
:100EF0002000A0000F30A100803110202000220827
:100F00002100D10009305107D20049308400850109
:100F10005208840777088000200022082100D100B1
:100F200005305107D200200022082100D3000830EC
:100F30005307D40049308400850152088407000813
:100F40002000A00049308400850121005408840756
:100F500020002008000287310319D72F21005008F4
:100F60002000A0000F30A1008031102020002208B6
:100F70002100D50005305507D600200022082100A9
:100F8000D70005305707D80049308400850158083C
:100F9000840700082000A00049308400850121005A
:100FA000560884072000200A80008731ED2F210099
:100FB00050082000A0000F30A10080311020200038
:100FC00022082100D10007305107D20049308400A7
:100FD000850152088407033080008831AE284930EB
:100FE0008400850152088407023000028831031D05
:100FF000AE2850082000A0000F30A1008031102042
:10100000200022082100D10009305107D2004930C8
:1010100084008501520884070008883103193828A4
:1010200050082000A0000F30A100803110202000C7
:1010300022082100D30009305307D40020002208E1
:101040002100D50009305507D600493084008501BC
:101050005608840700082000A0004930840085015C
:101060002100540884072000200380008831AE2826
:1010700050082000A0000F30A10080311020200077
:1010800022082100D10009305107D20049308400E4
:10109000850152088407770880002000220821007B
:1010A000D10005305107D200200022082100D300D2
:1010B00008305307D4004930840085015208840762
:1010C00000082000A0004930840085012100540858
:1010D0008407200020080002883103199828210085
:1010E00050082000A0000F30A10080311020200007
:1010F00022082100D50005305507D600200022081F
:101100002100D70005305707D800493084008501F9
:101110005808840700082000A00049308400850199
:101120002100560884072000200380008831AE2863
:10113000210050082000A0000F30A10080311020B5
:10114000200022082100D10007305107D200493089
:1011500084008501520884070430800020002208A2
:101160002100D1000C305107D200493084008501A4
:101170005208840700088A310319522A4930840032
:101180008501520884070330000288310319D128F1
:101190004930840085015208840704300002031D91
:1011A000D3288A31522A49308400850152088407A5
:1011B00000038931031D932950082000A0000F303F
:1011C000A10080311020200022082100D1000E3023
:1011D0005107D20049308400850152088407000875
:1011E000893103191B2950082000A0000F30A100ED
:1011F00080311020200022082100D3000E30530738
:10120000D400200022082100D5000E305507D6005A
:101210004930840085015608840700082000A0009A
:1012200049308400850121005408840720002003F0
:1012300080008A31522A50082000A0000F30A100FF
:1012400080311020200022082100D1000E305107EB
:10125000D200493084008501520884077708800055
:10126000200022082100D1000A305107D2002000BE
:1012700022082100D3000D305307D40049308400E8
:1012800085015208840700082000A000493084002E
:1012900085012100540884072000200800028931BC
:1012A00003197B29210050082000A0000F30A10065
:1012B00080311020200022082100D5000A30550777
:1012C000D600200022082100D7000A305707D80096
:1012D0004930840085015808840700082000A000D8
:1012E0004930840085012100560884072000200A27
:1012F000800089319129210050082000A0000F3082
:10130000A10080311020200022082100D1000C30E3
:101310005107D20049308400850152088407033008
:1013200080008A31522A493084008501520884079E
:10133000023000028A31031D522A50082000A0000A
:101340000F30A10080311020200022082100D100A0
:101350000E305107D20049308400850152088407BD
:10136000000889310319DC2950082000A0000F3043
:10137000A10080311020200022082100D3000E306F
:101380005307D400200022082100D5000E30550755
:10139000D6004930840085015608840700082000E3
:1013A000A0004930840085012100540884072000F2
:1013B000200380008A31522A50082000A0000F30FC
:1013C000A10080311020200022082100D1000E3021
:1013D0005107D200493084008501520884077708FC
:1013E0008000200022082100D1000A305107D200DD
:1013F000200022082100D3000D305307D4004930CB
:10140000840085015208840700082000A0004930AC
:101410008400850121005408840720002008000270
:101420008A3103193C2A210050082000A0000F3007
:10143000A10080311020200022082100D5000A30B0
:101440005507D600200022082100D7000A30570790
:10145000D80049308400850158088407000820001E
:10146000A00049308400850121005608840720002F
:10147000200380008A31522A210050082000A00059
:101480000F30A10080311020200022082100D1005F
:101490000C305107D200493084008501520884077E
:1014A000043080002100D00A033050028531031D32
:1014B000722D08007908031D742AFF30DA00FF300E
:1014C000DB00FF30DC00FF30DD00FF30DE00FF30EE
:1014D000DF00FF30E000FF30E100FF3085314D25B7
:1014E0000130F9008A3108007903031D882ADA01E6
:1014F000DB01FF30DC00DD01DE01FF30DF00E00159
:10150000E101FF3085314D250230F9008A310800B4
:1015100002307902031D9E2AFF30DA00DB01DC0174
:10152000FF30DD00DE01DF01FF30E000E1010030CF
:1015300085314D250330F9008A31080003307902E6
:10154000031DB42ADA01FF30DB00DC01DD01FF30CE
:10155000DE00DF01E001FF30E100003085314D2584
:101560000430F9008A31080004307902031DC42ACE
:10157000DA01DB01DC01DD01DE01DF01E001E10177
:10158000003085314D25F90108008031912021007E
:10159000CB00803191202100CC00803191202100AE
:1015A000CD004B084C028A310319E42A0318E42ABF
:1015B0004B084D020319E12A0318E12A4B08CE001B
:1015C000EF2A4D08CE00EF2A4C084D020319ED2AF0
:1015D0000318ED2A4C08CE00EF2A4D08CE004E0825
:1015E00076028B310319002B0318002B76084E026C
:1015F000CF00CB024F08CC024F08CC028B31082B16
:101600004E087602CF00CB074F08CC074F08CC0717
:101610004B0808008431EE248B3120002018132B56
:1016200021004910152B21004914491CCF2BC10161
:101630008A31C5222100C2004C08C3004D08C400F5
:1016400041082000A0000F30A100803110202000B0
:1016500022082100C500493084008501450884071F
:101660008001200022082100C50004304507C60083
:1016700049308400850146088407770880002000EF
:1016800022082100C50003304507C6004930840008
:1016900085014608840742088000200022082100B6
:1016A000C50002304507C600493084008501460860
:1016B000840701308000200022082100C500053089
:1016C0004507C6004930840085014608840780012B
:1016D000200022082100C50009304507C600493016
:1016E00084008501460884077708800020002208CE
:1016F0002100C50008304507C60049308400850137
:101700004608840743088000200022082100C50005
:1017100007304507C6004930840085014608840724
:1017200001308000200022082100C5000A30450752
:10173000C6004930840085014608840780012000E6
:1017400022082100C5000E304507C600493084003C
:1017500085014608840777088000200022082100C0
:10176000C5000D304507C600493084008501460894
:10177000840744088000200022082100C5000C30A6
:101780004507C600493084008501460884070130BA
:101790008000C10A033041028B31031D182BC101A7
:1017A00041082000A0000F30A1008031102020004F
:1017B00022082100C50002304507C60049308400D8
:1017C000850146088407033000028C31031D182C64
:1017D00041082000A0000F30A1008031102020001F
:1017E00022082100C70003304707C80049308400A1
:1017F0008501480884078001200022082100C500D7
:1018000004304507C6004930840085014608840736
:1018100077088000200022082100C500023045071B
:10182000C6004930840085014608840702308000E4
:10183000200022082100C50007304507C6004930B6
:101840008400850146088407033000028C31031DA3
:10185000592C41082000A0000F30A1008031102039
:10186000200022082100C70008304707C80049307F
:101870008400850148088407800120002208210097
:10188000C50009304507C600493084008501460877
:10189000840777088000200022082100C500073057
:1018A0004507C60049308400850146088407023098
:1018B0008000200022082100C5000C304507C6002A
:1018C00049308400850146088407033000028C31CA
:1018D000031D9A2C41082000A0000F30A100803188
:1018E0001020200022082100C7000D304707C80043
:1018F00049308400850148088407800120002208BF
:101900002100C5000E304507C6004930840085011E
:101910004608840777088000200022082100C500BF
:101920000C304507C600493084008501460884070D
:1019300002308000C10A033041028B31031DD02BDD
:10194000C1018A31C5222100C2004C08C3004D08E4
:10195000C40041082000A0000F30A10080311020F9
:10196000200022082100C50002304507C60049308A
:101970008400850146088407043000028C31031D71
:10198000F22C41082000A0000F30A100803110206F
:10199000200022082100C70003304707C800493053
:1019A000840085014808840742088000200022083E
:1019B0002100C50004304507C60049308400850178
:1019C0004608840777088000200022082100C5000F
:1019D00002304507C6004930840085014608840767
:1019E00001308000200022082100C5000730450793
:1019F000C60049308400850146088407043000028F
:101A00008D31031D342D41082000A0000F30A100AE
:101A100080311020200022082100C700083047072D
:101A2000C8004930840085014808840743088000C5
:101A3000200022082100C50009304507C6004930B2
:101A4000840085014608840777088000200022086A
:101A50002100C50007304507C600493084008501D4
:101A60004608840701308000200022082100C500BC
:101A70000C304507C60049308400850146088407BC
:101A8000043000028D31031D762D41082000A00096
:101A90000F30A10080311020200022082100C70053
:101AA0000D304707C8004930840085014808840785
:101AB00044088000200022082100C5000E304507A0
:101AC000C6004930840085014608840777088000F5
:101AD000200022082100C5000C304507C60049300F
:101AE000840085014608840701308000C10A033064
:101AF00041028C31031DA12C08008431EE248D316C
:101B000020002018862D21004010882D210040142F
:101B1000401C982D76082000D3007708D700D60106
:101B20000230D5007708DC007608DB000130DA00EF
:101B3000043020005502031DA42DD5017608EF00C6
:101B40007708F0000130EE0004305A02031DAF2D7B
:101B5000DA017608D6007708D7000130D5000430C6
:101B60006E02031DBA2DEE017608DB007708DC005B
:101B70000130DA0003305A02031DC42DDA01DB0103
:101B80007708DC000230DA0003306E02031DCE2D30
:101B9000EE01EF017708F0000230EE00033055024D
:101BA000031DD82DD501D6017708D7000230D50006
:101BB00008008431EE248D3120002018E22D210010
:101BC0003F10E42D21003F148D313F1CFA2D770882
:101BD0002000CD007608CC000130CB007708D20081
:101BE0007608D1000130D0007708D7007608D600FB
:101BF0000130D500033020004B028E31031D212E11
:101C00007708CD00CC010230CB007708D200D1019B
:101C10000230D0007708D700D6010230D50077080F
:101C2000DC007608DB000130DA007708E100760896
:101C3000E0000130DF007708E6007608E5000130BB
:101C4000E40003305A02031D462E7708DC00DB0156
:101C50000230DA007708E100E0010230DF007708A7
:101C6000E600E5010230E4007708EB007608EA00C0
:101C70000130E9007708F0007608EF000130EE004F
:101C80007708F5007608F4000130F30003306902AC
:101C9000031D6B2E7708EB00EA010230E90077089C
:101CA000F000EF010230EE007708F500F401023099
:101CB000F3007708CD007608CC000130CB00770820
:101CC000D2007608D1000130D0007708D70076081E
:101CD000D6000130D50008008431EE248E3120007A
:101CE0002018752E21003D10772E21003D143D1C3B
:101CF0009A2E8A31C5222100BA004C08BB004D083B
:101D0000BC0077082000CD0021003A082000CC005C
:101D10000130CB007708D20021003B082000D10021
:101D20000130D0007708D70021003C082000D60001
:101D30000130D500033020004B022100BD100319F3
:101D4000BD1403302000500221003D1103193D1540
:101D5000BD15BD183D1DBD110330200055022100E9
:101D60003D1203193D16BD16BD193D1EBD128E3123
:101D7000BD1EEA2E8A31C5222100BA004C08BB00E4
:101D80004D08BC0077082000CD00CC010230CB000C
:101D90007708D200D1010230D0007708D700D601F1
:101DA0000230D5007708DC0021003A082000DB0073
:101DB0000130DA007708E10021003B082000E00054
:101DC0000130DF007708E60021003C082000E50034
:101DD0000130E400033020005A0221003D130319B2
:101DE0003D17033020005F022100BD130319BD170A
:101DF0003E143D1BBD1F3E10033020006402210035
:101E0000BE100319BE143E153E18BE1C3E118F3184
:101E10003E1D3A2F8A31C5222100BA004C08BB0072
:101E20004D08BC0077082000DC00DB010230DA003E
:101E30007708E100E0010230DF007708E600E50105
:101E40000230E4007708EB0021003A082000EA00A5
:101E50000130E9007708F00021003B082000EF0086
:101E60000130EE007708F50021003C082000F40066
:101E70000130F3000330200069022100BE11031974
:101E8000BE15033020006E0221003E1203193E16DB
:101E9000BE16BE193E1EBE12033020007302210082
:101EA0003E1303193E17BE17BE1A3E1FBE138F31D5
:101EB000BE1F8A2F8A31C5222100BA004C08BB0000
:101EC0004D08BC0077082000EB00EA010230E90071
:101ED0007708F000EF010230EE007708F500F4011A
:101EE0000230F3007708CD0021003A082000CC0032
:101EF0000130CB007708D20021003B082000D10040
:101F00000130D0007708D70021003C082000D6001F
:101F10000130D50008008431EE248F3120002018D4
:101F2000942F21003810962F21003814381C9F2F31
:101F300077082000CD007608CC000130CB000330BC
:101F400020004B02031DB52FCC017708CD000230D5
:101F5000CB007608D1007708D2000130D000760897
:101F6000DB007708DC000130DA0003305002031D8B
:101F7000CA2FD1017708D2000230D0007608D600EF
:101F80007708D7000130D5007608E0007708E10037
:101F90000130DF0003305502031DD92FD601770829
:101FA000D7000230D5007608E5007708E60001305A
:101FB000E40003305A02031DEE2FDB017708DC003A
:101FC0000230DA007608E0007708E1000130DF0037
:101FD0007608EA007708EB000130E90003305F0281
:101FE0009031031D0428E0017708E1000230DF0092
:101FF0007608E5007708E6000130E4007608EF0097
:102000007708F0000130EE0003306402031D13284E
:10201000E5017708E6000230E4007608F40077086E
:10202000F5000130F30003306902031D2828EA019E
:102030007708EB000230E9007608EF007708F0003F
:102040000130EE007608CC007708CD000130CB00DF
:1020500003306E02031D3D28EF017708F0000230C7
:10206000EE007608F4007708F5000130F3007608FA
:10207000D1007708D2000130D00003307302031D75
:102080004C28F4017708F5000230F3007608D600FA
:102090007708D7000130D50008008431EE24903154
:1020A0002000201856282100311058282100311412
:1020B000311C632877082000CD00FF30CC000130B0
:1020C000CB000130F8007808031D68289231080021
:1020D0007803031D7428033020004B029231031D46
:1020E0004D2A0230F800080002307802031D8F28C4
:1020F000FC302000DB007708DC000130DA006A30B9
:10210000E0007708E1000130DF001030E5007708DB
:10211000E6000130E4000330F8009231080003309B
:102120007802031DB628033020005A022100311323
:1021300003193117033020005F022100B113031986
:10214000B1173214311BB11F32100330200064026A
:102150002100B2100319B21432153218B21C321118
:102160009231321D4D2A0430F80008000430780204
:10217000031DD128ED302000EA007708EB00013084
:10218000E900FE30EF007708F0000130EE000E307D
:10219000F4007708F5000130F3000530F8009231C3
:1021A000080005307802031DF8280330200069027A
:1021B0002100B2120319B216033020006E02210072
:1021C000321303193217B217B21A321FB213033087
:1021D000200073022100331003193314B314B21B0F
:1021E000331CB3109231B31C4D2A0630F80008009E
:1021F000063078029131031D0D292000CC017708AB
:10220000CD000230CB00FF30D1007708D200013082
:10221000D0000730F8009231080007307802031D23
:102220002929043020004B022100331203193316F0
:102230000330200050022100B3120319B3163317E4
:10224000331AB31E33139231331F4D2A0830F8006E
:10225000080008307802031D42292000DB017708BE
:10226000DC000230DA00E0017708E1000230DF0034
:10227000FF30E5007708E6000130E4000930F8009F
:102280009231080009307802031D692904302000CA
:102290005A022100B4100319B414043020005F0264
:1022A0002100341103193415B415B418341DB411B8
:1022B0000330200064022100341203193416B416CE
:1022C000B419341EB4129231B41E4D2A0A30F800EB
:1022D00008000A307802031D8429FE302000EA003D
:1022E0007708EB000130E9000E30EF007708F000CE
:1022F0000230EE00F330F4007708F5000130F3000F
:102300000B30F800923108000B307802031DAB2926
:102310000330200069022100351003193514043000
:1023200020006E022100B5100319B51435153518BB
:10233000B51C35110330200073022100B5110319BB
:10234000B51535163519B51D35129231351E4D2A84
:102350000C30F80008000C307802031DBF29FF3054
:102360002000CC007708CD000130CB00D1017708E8
:10237000D2000230D0000D30F800923108000D304C
:102380007802031DCC29033020004B029231031D3B
:102390004D2A0E30F80008000E307802031DE729A0
:1023A000FC302000DB007708DC000130DA006A3006
:1023B000E0007708E1000130DF001030E500770829
:1023C000E6000230E4000F30F800923108000F30D0
:1023D00078029231031D0E2A033020005A02210098
:1023E000361103193615033020005F022100B611A3
:1023F0000319B61536163619B61D361204302000EC
:1024000064022100B6120319B6163617361AB61E24
:102410003613361F4D2A1030F800080010307802AD
:10242000031D282AED302000EA007708EB00023077
:10243000E900FE30EF007708F0000130EE000E30CA
:10244000F4007708F5000230F3001130F8000800BE
:1024500011307802031D4D2A04302000690221004A
:10246000B7100319B714033020006E022100371192
:1024700003193715B715B718371DB71104302000E9
:1024800073022100371203193716B716B719371E12
:10249000B712B71E4D2A0630F80008008431EE242A
:1024A000923120002018572A21002F10592A21008C
:1024B0002F142F1C702A77082000CD007608CC003E
:1024C0000130CB000A307707DC007608DB000130F2
:1024D000DA000A307707EB007608EA000130E900FD
:1024E000033020004B02031D802ACC017708CD0069
:1024F0000230CB007608D1007708D2000130D0003E
:1025000003305002031D8F2AD1017708D200023018
:10251000D0007608D6007708D7000130D500033008
:102520005502031D9E2AD6017708D7000230D50038
:102530007608CC007708CD000130CB0003305A027A
:10254000031DAF2ADB010A307707DC000230DA0016
:102550007608E0000A307707E1000130DF00033041
:102560005F02031DC02AE0010A307707E100023054
:10257000DF007608E5000A307707E6000130E40066
:1025800003306402031DD12AE5010A307707E60013
:102590000230E4007608DB000A307707DC00013007
:1025A000DA0003306902031DE22AEA0114307707DA
:1025B000EB000230E9007608EF0014307707F000F6
:1025C0000130EE0003306E02031DF32AEF011430D8
:1025D0007707F0000230EE007608F4001430770739
:1025E000F5000130F300033073029331031D052B16
:1025F000F40114307707F5000230F3007608EA00A2
:1026000014307707EB000130E90008009917873094
:10261000190570389900FC309905951723008C0135
:102620008E0121009D019E012200910192019301E2
:10263000940121000C12392B28001E1187301E0531
:1026400008389E00FC301E0503389E007C309D003B
:102650002000931121009315A51028001E150B17BB
:102660008B1708008331931DD02B93112100A514E3
:10267000D02B20003030A000F830A1006E30A20036
:102680009331A20B412B9331A10B3E2B9331A00B25
:102690003C2B20000330A0009331A00B4D2B0000F9
:1026A0000000003083312F23FE00AB307E029331D7
:1026B00003198E2BAB302100E90000308331382321
:1026C000E130FA00AC30FB007A082100E90001306B
:1026D000833138237B082100E9000230833138231D
:1026E0007A082100ED007B08EE0080311E20FF30CB
:1026F000F6002100E9000430833138230730F70069
:102700002100E9000530833138230130FC0021002D
:10271000E9000330833138239331BC2B01308331FE
:102720002F23FA00023083312F23FB007A08210087
:10273000ED007B08EE0080311E2080318A202000D1
:102740002008FA002108FB007A082100E900013086
:10275000833138237B082100E9000230833138239C
:10276000043083312F23F600053083312F23F70007
:10277000033083312F23FC0083316B2383315923B2
:1027800093311C238031A0208031F0202100A00152
:10279000A101A201A3012511A511251684311F2431
:1027A000F801F9017C089331031DE22B2100200878
:1027B00021049431031D492C63008830A00013309C
:1027C000A100492C7C03031DE92B8D317D2594311B
:1027D000492C02307C02031DF12B8D31D925943117
:1027E000492C03307C02031DF92B8F318B27943148
:1027F000492C04307C029431031D022C90314D2071
:102800009431492C05307C029431031D222C76082A
:10281000031D0C2C0130F60076082100DA00760842
:10282000DB007608DC007608DD007608DE0076083E
:10283000DF007608E0007608E100760885314D2556
:102840009431492C07307C02031D2A2C8B310A233A
:102850009431492C08307C02031D322C8E316C26B9
:102860009431492C09307C02031D3A2C92314E22BE
:102870009431492C06307C02031D492C210020088C
:102880002104031D492CD030A0000730A1008A315B
:102890005A2294312100A51C602CA5102008210487
:1028A0000319562CA003200A0319A10322082304AC
:1028B00003195E2CA203220A0319A3038531712593
:1028C0008031F720943120002018692C2100A712B4
:1028D0006B2C2100A716813109219431200020188A
:1028E000742C21002713762C21002717A713A71E6D
:1028F000271BA7179331A71FD22B7C08FD00103090
:10290000200048029431031D972CFA3076022100F2
:10291000A810031D031CA8142815251AA81C28118B
:102920009531281DF82D0530F607A515F82D113025
:102930004802031DAD2C0530760221002812031D2C
:1029400003182816A816251A281EA8129531A81EA5
:10295000F82D0530F602A515F82D20304802031D8C
:10296000C02C77082100A8170319A8132914251AC9
:10297000A81F29109531291CF82DF703A515F82D4E
:1029800021304802031DD42C323077022100291156
:10299000031D2915A915251A291DA9119531A91D50
:1029A000F82DF70AA515F82D4808031DDE2C9531E2
:1029B0002100251EF82D0530FC00F82D4803031DCD
:1029C000E82C95312100251EF82D0130FC00F82D52
:1029D00002304802031DF32C95312100251EF82DED
:1029E0000230FC00F82D03304802031DFE2C953107
:1029F0002100251EF82D0330FC00F82D043048027C
:102A00009531031D252D210022082304AA14031D3E
:102A1000AA102A11251D0F2D251C102D112D25184A
:102A20002A15AA11AA1C2A19AA152A16251AAA1D9E
:102A30002A122A1E212D251125182515F8010430EA
:102A4000FC00C830A200A301F82D05304802031D88
:102A50002F2D2100251EF82D0730FC00F82D063003
:102A60004802031D392D2100251EF82D0830FC00D9
:102A7000F82D07304802031D432D2100251EF82D97
:102A80000930FC00F82D08304802031D692D210093
:102A900022082304AB14031DAB102B11251D532D4D
:102AA000251C542D552D25182B15AB11AB1C2B199E
:102AB000AB152B16251AAB1D2B122B1E652D2511C0
:102AC00025182515F9010630FC00C830A200A30125
:102AD000F82D0D304802031D932D210022082304F8
:102AE0002B17031D2B13AB13251D792D251C7A2DB8
:102AF0007B2D2518AB172C102B1FAB1B2C14AC14E3
:102B0000251A2C1CAC10AC1C8F2D25112518251551
:102B1000FF30F6000730F7000130FC00A515C83083
:102B2000A200A301F82D0C304802031DF82D21004E
:102B300022082304AC15031DAC112C12251DA32D56
:102B4000251CA42DA52D25182C16AC12AC1D2C1A55
:102B5000AC16AC1EF52D251125182515251EE52DC5
:102B600084311F2495312100A51DDD2D80318A205F
:102B700020002008FA002108FB007A082100E90063
:102B80000130833138237B082100E9000230833192
:102B9000382376082100E900043083313823770890
:102BA0002100E9000530833138237C082100E90049
:102BB0000330833138232100A51125128830A0006D
:102BC0001330A100FC019531F52D043083312F2302
:102BD000F600053083312F23F700033083312F2394
:102BE000FC002100A001A1012516C830A200A3010C
:102BF0007D087C0293310319D22B84311F242100DC
:062C0000A5159331D22B53
:020000040001F9
:02000E00840963
:02001000FF1ED1
:00000001FF
